Archive member included because of file (symbol)

/opt/toolchains/sega/m68k-elf/lib/libpcm.a(pcm.o)
                              module.o (pcm_load_samples)
/opt/toolchains/sega/m68k-elf/lib/libpcm.a(pcm-io.o)
                              /opt/toolchains/sega/m68k-elf/lib/libpcm.a(pcm.o) (pcm_lcf)
/opt/toolchains/sega/m68k-elf/m68k-elf/lib/libc.a(lib_a-malloc.o)
                              module.o (malloc)
/opt/toolchains/sega/m68k-elf/m68k-elf/lib/libc.a(lib_a-mallocr.o)
                              /opt/toolchains/sega/m68k-elf/m68k-elf/lib/libc.a(lib_a-malloc.o) (_malloc_r)
/opt/toolchains/sega/m68k-elf/m68k-elf/lib/libc.a(lib_a-memcmp.o)
                              main.o (memcmp)
/opt/toolchains/sega/m68k-elf/m68k-elf/lib/libc.a(lib_a-memcpy.o)
                              main.o (memcpy)
/opt/toolchains/sega/m68k-elf/m68k-elf/lib/libc.a(lib_a-memset.o)
                              main.o (memset)
/opt/toolchains/sega/m68k-elf/m68k-elf/lib/libc.a(lib_a-mlock.o)
                              /opt/toolchains/sega/m68k-elf/m68k-elf/lib/libc.a(lib_a-mallocr.o) (__malloc_lock)
/opt/toolchains/sega/m68k-elf/m68k-elf/lib/libc.a(lib_a-rand.o)
                              module.o (rand)
/opt/toolchains/sega/m68k-elf/m68k-elf/lib/libc.a(lib_a-sbrkr.o)
                              /opt/toolchains/sega/m68k-elf/m68k-elf/lib/libc.a(lib_a-mallocr.o) (_sbrk_r)
/opt/toolchains/sega/m68k-elf/m68k-elf/lib/libc.a(lib_a-sprintf.o)
                              main.o (sprintf)
/opt/toolchains/sega/m68k-elf/m68k-elf/lib/libc.a(lib_a-strcat.o)
                              main.o (strcat)
/opt/toolchains/sega/m68k-elf/m68k-elf/lib/libc.a(lib_a-strcpy.o)
                              main.o (strcpy)
/opt/toolchains/sega/m68k-elf/m68k-elf/lib/libc.a(lib_a-strlen.o)
                              cdfh.o (strlen)
/opt/toolchains/sega/m68k-elf/m68k-elf/lib/libc.a(lib_a-strncpy.o)
                              cdfh.o (strncpy)
/opt/toolchains/sega/m68k-elf/m68k-elf/lib/libc.a(lib_a-svfprintf.o)
                              /opt/toolchains/sega/m68k-elf/m68k-elf/lib/libc.a(lib_a-sprintf.o) (_svfprintf_r)
/opt/toolchains/sega/m68k-elf/m68k-elf/lib/libc.a(lib_a-dtoa.o)
                              /opt/toolchains/sega/m68k-elf/m68k-elf/lib/libc.a(lib_a-svfprintf.o) (_dtoa_r)
/opt/toolchains/sega/m68k-elf/m68k-elf/lib/libc.a(lib_a-freer.o)
                              /opt/toolchains/sega/m68k-elf/m68k-elf/lib/libc.a(lib_a-malloc.o) (_free_r)
/opt/toolchains/sega/m68k-elf/m68k-elf/lib/libc.a(lib_a-impure.o)
                              /opt/toolchains/sega/m68k-elf/m68k-elf/lib/libc.a(lib_a-malloc.o) (_impure_ptr)
/opt/toolchains/sega/m68k-elf/m68k-elf/lib/libc.a(lib_a-locale.o)
                              /opt/toolchains/sega/m68k-elf/m68k-elf/lib/libc.a(lib_a-svfprintf.o) (_localeconv_r)
/opt/toolchains/sega/m68k-elf/m68k-elf/lib/libc.a(lib_a-memchr.o)
                              /opt/toolchains/sega/m68k-elf/m68k-elf/lib/libc.a(lib_a-svfprintf.o) (memchr)
/opt/toolchains/sega/m68k-elf/m68k-elf/lib/libc.a(lib_a-mprec.o)
                              /opt/toolchains/sega/m68k-elf/m68k-elf/lib/libc.a(lib_a-dtoa.o) (_Balloc)
/opt/toolchains/sega/m68k-elf/m68k-elf/lib/libc.a(lib_a-reent.o)
                              /opt/toolchains/sega/m68k-elf/m68k-elf/lib/libc.a(lib_a-sbrkr.o) (errno)
/opt/toolchains/sega/m68k-elf/m68k-elf/lib/libc.a(lib_a-s_fpclassify.o)
                              /opt/toolchains/sega/m68k-elf/m68k-elf/lib/libc.a(lib_a-svfprintf.o) (__fpclassifyd)
/opt/toolchains/sega/m68k-elf/m68k-elf/lib/libc.a(lib_a-strcmp.o)
                              /opt/toolchains/sega/m68k-elf/m68k-elf/lib/libc.a(lib_a-locale.o) (strcmp)
/opt/toolchains/sega/m68k-elf/m68k-elf/lib/libc.a(lib_a-svfiprintf.o)
                              /opt/toolchains/sega/m68k-elf/m68k-elf/lib/libc.a(lib_a-svfprintf.o) (__ssprint_r)
/opt/toolchains/sega/m68k-elf/m68k-elf/lib/libc.a(lib_a-callocr.o)
                              /opt/toolchains/sega/m68k-elf/m68k-elf/lib/libc.a(lib_a-mprec.o) (_calloc_r)
/opt/toolchains/sega/m68k-elf/m68k-elf/lib/libc.a(lib_a-memmove.o)
                              /opt/toolchains/sega/m68k-elf/m68k-elf/lib/libc.a(lib_a-svfiprintf.o) (memmove)
/opt/toolchains/sega/m68k-elf/m68k-elf/lib/libc.a(lib_a-reallocr.o)
                              /opt/toolchains/sega/m68k-elf/m68k-elf/lib/libc.a(lib_a-svfiprintf.o) (_realloc_r)
/opt/toolchains/sega/m68k-elf/lib/gcc/m68k-elf/4.6.2/libgcc.a(_mulsi3.o)
                              module.o (__mulsi3)
/opt/toolchains/sega/m68k-elf/lib/gcc/m68k-elf/4.6.2/libgcc.a(_udivsi3.o)
                              /opt/toolchains/sega/m68k-elf/m68k-elf/lib/libc.a(lib_a-svfprintf.o) (__udivsi3)
/opt/toolchains/sega/m68k-elf/lib/gcc/m68k-elf/4.6.2/libgcc.a(_divsi3.o)
                              /opt/toolchains/sega/m68k-elf/m68k-elf/lib/libc.a(lib_a-svfprintf.o) (__divsi3)
/opt/toolchains/sega/m68k-elf/lib/gcc/m68k-elf/4.6.2/libgcc.a(_umodsi3.o)
                              /opt/toolchains/sega/m68k-elf/m68k-elf/lib/libc.a(lib_a-svfprintf.o) (__umodsi3)
/opt/toolchains/sega/m68k-elf/lib/gcc/m68k-elf/4.6.2/libgcc.a(_modsi3.o)
                              /opt/toolchains/sega/m68k-elf/m68k-elf/lib/libc.a(lib_a-svfprintf.o) (__modsi3)
/opt/toolchains/sega/m68k-elf/lib/gcc/m68k-elf/4.6.2/libgcc.a(_double.o)
                              /opt/toolchains/sega/m68k-elf/m68k-elf/lib/libc.a(lib_a-dtoa.o) (__adddf3)
/opt/toolchains/sega/m68k-elf/lib/gcc/m68k-elf/4.6.2/libgcc.a(_floatex.o)
                              /opt/toolchains/sega/m68k-elf/lib/gcc/m68k-elf/4.6.2/libgcc.a(_double.o) (_fpCCR)
/opt/toolchains/sega/m68k-elf/lib/gcc/m68k-elf/4.6.2/libgcc.a(_eqdf2.o)
                              /opt/toolchains/sega/m68k-elf/m68k-elf/lib/libc.a(lib_a-svfprintf.o) (__eqdf2)
/opt/toolchains/sega/m68k-elf/lib/gcc/m68k-elf/4.6.2/libgcc.a(_nedf2.o)
                              /opt/toolchains/sega/m68k-elf/m68k-elf/lib/libc.a(lib_a-svfprintf.o) (__nedf2)
/opt/toolchains/sega/m68k-elf/lib/gcc/m68k-elf/4.6.2/libgcc.a(_gtdf2.o)
                              /opt/toolchains/sega/m68k-elf/m68k-elf/lib/libc.a(lib_a-dtoa.o) (__gtdf2)
/opt/toolchains/sega/m68k-elf/lib/gcc/m68k-elf/4.6.2/libgcc.a(_gedf2.o)
                              /opt/toolchains/sega/m68k-elf/m68k-elf/lib/libc.a(lib_a-dtoa.o) (__gedf2)
/opt/toolchains/sega/m68k-elf/lib/gcc/m68k-elf/4.6.2/libgcc.a(_ltdf2.o)
                              /opt/toolchains/sega/m68k-elf/m68k-elf/lib/libc.a(lib_a-svfprintf.o) (__ltdf2)
/opt/toolchains/sega/m68k-elf/lib/gcc/m68k-elf/4.6.2/libgcc.a(_muldi3.o)
                              /opt/toolchains/sega/m68k-elf/m68k-elf/lib/libc.a(lib_a-rand.o) (__muldi3)
/opt/toolchains/sega/m68k-elf/lib/gcc/m68k-elf/4.6.2/libgcc.a(fpgnulib.o)
                              /opt/toolchains/sega/m68k-elf/m68k-elf/lib/libc.a(lib_a-dtoa.o) (__floatunsidf)
/opt/toolchains/sega/m68k-elf/lib/gcc/m68k-elf/4.6.2/libgcc.a(xfgnulib.o)
                              /opt/toolchains/sega/m68k-elf/m68k-elf/lib/libc.a(lib_a-svfprintf.o) (__truncxfdf2)
/opt/toolchains/sega/m68k-elf/m68k-elf/lib/libnosys.a(sbrk.o)
                              /opt/toolchains/sega/m68k-elf/m68k-elf/lib/libc.a(lib_a-sbrkr.o) (sbrk)

Allocating common symbols
Common symbol       size              file

errno               0x4               /opt/toolchains/sega/m68k-elf/m68k-elf/lib/libc.a(lib_a-reent.o)
gDirTable           0x10000           main.o
voices              0x70              module.o

Memory Configuration

Name             Origin             Length             Attributes
ram              0x00008000         0x00078000         xw
*default*        0x00000000         0xffffffff

Linker script and memory map

LOAD crt0.o
LOAD main.o
LOAD module.o
LOAD cdfh.o
LOAD hw_md.o
LOAD /opt/toolchains/sega/m68k-elf/lib/libpcm.a
LOAD /opt/toolchains/sega/m68k-elf/m68k-elf/lib/libc.a
LOAD /opt/toolchains/sega/m68k-elf/lib/gcc/m68k-elf/4.6.2/libgcc.a
LOAD /opt/toolchains/sega/m68k-elf/m68k-elf/lib/libnosys.a
                0x00000000                __DYNAMIC = 0x0
                0x00080000                PROVIDE (__stack, 0x80000)

.text           0x00008000     0xd2b0
                0x00008000                __text_start = .
 *(.text)
 .text          0x00008000       0x4c crt0.o
                0x00008000                _start
 .text          0x0000804c      0x7a8 main.o
                0x0000804c                getCurrDir
                0x000080ea                main
 .text          0x000087f4     0x1d70 module.o
                0x00008bae                InitMOD
                0x0000927a                StartMOD
                0x000092ba                PauseMOD
                0x0000934a                StopMOD
                0x0000936a                ExitMOD
                0x000093a8                WaitMOD
                0x000093c0                CheckMOD
                0x000093d2                VolumeMOD
                0x000093ec                JumpMOD
                0x00009412                TimeScaleMOD
                0x00009436                PlayMOD
 .text          0x0000a564      0x34a cdfh.o
                0x0000a70c                cd_handle_from_offset
                0x0000a75e                cd_handle_from_name
                0x0000a89c                delete_cd_handle
 *fill*         0x0000a8ae        0x2 00
 .text          0x0000a8b0     0x19cc hw_md.o
                0x0000a8b0                init_cd
                0x0000a8cc                read_cd
                0x0000a8ee                set_cwd
                0x0000a908                first_dir_sec
                0x0000a91e                next_dir_sec
                0x0000a934                find_dir_entry
                0x0000a94e                next_dir_entry
                0x0000a964                load_file
                0x0000a9c0                do_md_cmd0
                0x0000a9ce                do_md_cmd1
                0x0000a9e2                do_md_cmd2
                0x0000a9fc                do_md_cmd3
                0x0000aa1c                do_md_cmd4
                0x0000aa42                send_md_cmd0
                0x0000aa48                send_md_cmd1
                0x0000aa54                send_md_cmd2
                0x0000aa66                send_md_cmd3
                0x0000aa7e                send_md_cmd4
                0x0000aac0                wait_md_cmd
                0x0000aacc                switch_banks
                0x0000aadc                sub_delay
                0x0000aafc                init_hardware
 .text          0x0000c27c      0x250 /opt/toolchains/sega/m68k-elf/lib/libpcm.a(pcm.o)
                0x0000c320                pcm_load_samples
                0x0000c376                pcm_next_block
                0x0000c38e                pcm_reset
                0x0000c40a                pcm_set_ctrl
                0x0000c41a                pcm_set_off
                0x0000c43e                pcm_set_on
                0x0000c462                pcm_set_start
                0x0000c478                pcm_set_loop
                0x0000c49e                pcm_set_env
                0x0000c4ae                pcm_set_pan
 .text          0x0000c4cc      0x12c /opt/toolchains/sega/m68k-elf/lib/libpcm.a(pcm-io.o)
                0x0000c4cc                pcm_lcf
                0x0000c4f2                pcm_delay
                0x0000c4fa                pcm_set_period
                0x0000c526                pcm_set_freq
                0x0000c554                pcm_set_timer
                0x0000c576                pcm_stop_timer
                0x0000c592                pcm_start_timer
 .text          0x0000c5f8       0x32 /opt/toolchains/sega/m68k-elf/m68k-elf/lib/libc.a(lib_a-malloc.o)
                0x0000c5f8                malloc
                0x0000c610                free
 *fill*         0x0000c62a        0x2 00
 .text          0x0000c62c      0x73c /opt/toolchains/sega/m68k-elf/m68k-elf/lib/libc.a(lib_a-mallocr.o)
                0x0000c62c                _malloc_r
 .text          0x0000cd68       0x8c /opt/toolchains/sega/m68k-elf/m68k-elf/lib/libc.a(lib_a-memcmp.o)
                0x0000cd68                memcmp
 .text          0x0000cdf4       0x6e /opt/toolchains/sega/m68k-elf/m68k-elf/lib/libc.a(lib_a-memcpy.o)
                0x0000cdf4                memcpy
 *fill*         0x0000ce62        0x2 00
 .text          0x0000ce64       0x72 /opt/toolchains/sega/m68k-elf/m68k-elf/lib/libc.a(lib_a-memset.o)
                0x0000ce64                memset
 *fill*         0x0000ced6        0x2 00
 .text          0x0000ced8       0x10 /opt/toolchains/sega/m68k-elf/m68k-elf/lib/libc.a(lib_a-mlock.o)
                0x0000ced8                __malloc_lock
                0x0000cee0                __malloc_unlock
 .text          0x0000cee8       0x62 /opt/toolchains/sega/m68k-elf/m68k-elf/lib/libc.a(lib_a-rand.o)
                0x0000cee8                srand
                0x0000cf00                rand
 *fill*         0x0000cf4a        0x2 00
 .text          0x0000cf4c       0x32 /opt/toolchains/sega/m68k-elf/m68k-elf/lib/libc.a(lib_a-sbrkr.o)
                0x0000cf4c                _sbrk_r
 *fill*         0x0000cf7e        0x2 00
 .text          0x0000cf80       0x9a /opt/toolchains/sega/m68k-elf/m68k-elf/lib/libc.a(lib_a-sprintf.o)
                0x0000cf80                _sprintf_r
                0x0000cfcc                sprintf
 *fill*         0x0000d01a        0x2 00
 .text          0x0000d01c       0x7e /opt/toolchains/sega/m68k-elf/m68k-elf/lib/libc.a(lib_a-strcat.o)
                0x0000d01c                strcat
 *fill*         0x0000d09a        0x2 00
 .text          0x0000d09c       0x1a /opt/toolchains/sega/m68k-elf/m68k-elf/lib/libc.a(lib_a-strcpy.o)
                0x0000d09c                strcpy
 *fill*         0x0000d0b6        0x2 00
 .text          0x0000d0b8       0x1a /opt/toolchains/sega/m68k-elf/m68k-elf/lib/libc.a(lib_a-strlen.o)
                0x0000d0b8                strlen
 *fill*         0x0000d0d2        0x2 00
 .text          0x0000d0d4       0x86 /opt/toolchains/sega/m68k-elf/m68k-elf/lib/libc.a(lib_a-strncpy.o)
                0x0000d0d4                strncpy
 *fill*         0x0000d15a        0x2 00
 .text          0x0000d15c     0x1918 /opt/toolchains/sega/m68k-elf/m68k-elf/lib/libc.a(lib_a-svfprintf.o)
                0x0000d15c                _svfprintf_r
 .text          0x0000ea74     0x181c /opt/toolchains/sega/m68k-elf/m68k-elf/lib/libc.a(lib_a-dtoa.o)
                0x0000ec58                _dtoa_r
 .text          0x00010290      0x3d4 /opt/toolchains/sega/m68k-elf/m68k-elf/lib/libc.a(lib_a-freer.o)
                0x00010290                _malloc_trim_r
                0x0001037a                _free_r
 .text          0x00010664        0x0 /opt/toolchains/sega/m68k-elf/m68k-elf/lib/libc.a(lib_a-impure.o)
 .text          0x00010664       0xd0 /opt/toolchains/sega/m68k-elf/m68k-elf/lib/libc.a(lib_a-locale.o)
                0x00010664                _setlocale_r
                0x000106ca                __locale_charset
                0x000106d8                __locale_mb_cur_max
                0x000106e6                __locale_msgcharset
                0x000106f4                __locale_cjk_lang
                0x000106fe                _localeconv_r
                0x0001070c                setlocale
                0x00010726                localeconv
 .text          0x00010734       0xb0 /opt/toolchains/sega/m68k-elf/m68k-elf/lib/libc.a(lib_a-memchr.o)
                0x00010734                memchr
 .text          0x000107e4      0xdec /opt/toolchains/sega/m68k-elf/m68k-elf/lib/libc.a(lib_a-mprec.o)
                0x000107e4                _Balloc
                0x00010882                _Bfree
                0x000108ac                __multadd
                0x0001098e                __s2b
                0x00010a52                __hi0bits
                0x00010ab6                __lo0bits
                0x00010b3a                __i2b
                0x00010b5c                __multiply
                0x00010e0a                __pow5mult
                0x00010ee0                __lshift
                0x00010fbc                __mcmp
                0x00011016                __mdiff
                0x00011180                __ulp
                0x000111dc                __b2d
                0x000112d6                __d2b
                0x000113ec                __ratio
                0x0001148c                _mprec_log10
                0x000114ee                __copybits
                0x0001154c                __any_on
 .text          0x000115d0      0x1b0 /opt/toolchains/sega/m68k-elf/m68k-elf/lib/libc.a(lib_a-reent.o)
                0x000115d0                cleanup_glue
                0x00011606                _reclaim_reent
                0x00011704                _wrapup_reent
 .text          0x00011780       0x86 /opt/toolchains/sega/m68k-elf/m68k-elf/lib/libc.a(lib_a-s_fpclassify.o)
                0x00011780                __fpclassifyd
 *fill*         0x00011806        0x2 00
 .text          0x00011808       0xa4 /opt/toolchains/sega/m68k-elf/m68k-elf/lib/libc.a(lib_a-strcmp.o)
                0x00011808                strcmp
 .text          0x000118ac      0xd06 /opt/toolchains/sega/m68k-elf/m68k-elf/lib/libc.a(lib_a-svfiprintf.o)
                0x000118ac                __ssprint_r
                0x00011a34                _svfiprintf_r
 *fill*         0x000125b2        0x2 00
 .text          0x000125b4       0xc4 /opt/toolchains/sega/m68k-elf/m68k-elf/lib/libc.a(lib_a-callocr.o)
                0x000125b4                _calloc_r
 .text          0x00012678       0xe2 /opt/toolchains/sega/m68k-elf/m68k-elf/lib/libc.a(lib_a-memmove.o)
                0x00012678                memmove
 *fill*         0x0001275a        0x2 00
 .text          0x0001275c      0x644 /opt/toolchains/sega/m68k-elf/m68k-elf/lib/libc.a(lib_a-reallocr.o)
                0x0001275c                _realloc_r
 .text          0x00012da0       0x22 /opt/toolchains/sega/m68k-elf/lib/gcc/m68k-elf/4.6.2/libgcc.a(_mulsi3.o)
                0x00012da0                __mulsi3
 *fill*         0x00012dc2        0x2 00
 .text          0x00012dc4       0x5c /opt/toolchains/sega/m68k-elf/lib/gcc/m68k-elf/4.6.2/libgcc.a(_udivsi3.o)
                0x00012dc4                __udivsi3
 .text          0x00012e20       0x2e /opt/toolchains/sega/m68k-elf/lib/gcc/m68k-elf/4.6.2/libgcc.a(_divsi3.o)
                0x00012e20                __divsi3
 *fill*         0x00012e4e        0x2 00
 .text          0x00012e50       0x2e /opt/toolchains/sega/m68k-elf/lib/gcc/m68k-elf/4.6.2/libgcc.a(_umodsi3.o)
                0x00012e50                __umodsi3
 *fill*         0x00012e7e        0x2 00
 .text          0x00012e80       0x2e /opt/toolchains/sega/m68k-elf/lib/gcc/m68k-elf/4.6.2/libgcc.a(_modsi3.o)
                0x00012e80                __modsi3
 *fill*         0x00012eae        0x2 00
 .text          0x00012eb0      0x9cc /opt/toolchains/sega/m68k-elf/lib/gcc/m68k-elf/4.6.2/libgcc.a(_double.o)
                0x00012f0a                __subdf3
                0x00012f10                __adddf3
                0x000132a6                __muldf3
                0x00013454                __divdf3
                0x000136c8                __negdf2
                0x00013726                __cmpdf2_internal
                0x000137f6                __cmpdf2
 .text          0x0001387c       0x6a /opt/toolchains/sega/m68k-elf/lib/gcc/m68k-elf/4.6.2/libgcc.a(_floatex.o)
                0x0001387c                __clear_sticky_bit
                0x0001388a                $_exception_handler
 *fill*         0x000138e6        0x2 00
 .text          0x000138e8       0x22 /opt/toolchains/sega/m68k-elf/lib/gcc/m68k-elf/4.6.2/libgcc.a(_eqdf2.o)
                0x000138e8                __eqdf2
 *fill*         0x0001390a        0x2 00
 .text          0x0001390c       0x22 /opt/toolchains/sega/m68k-elf/lib/gcc/m68k-elf/4.6.2/libgcc.a(_nedf2.o)
                0x0001390c                __nedf2
 *fill*         0x0001392e        0x2 00
 .text          0x00013930       0x22 /opt/toolchains/sega/m68k-elf/lib/gcc/m68k-elf/4.6.2/libgcc.a(_gtdf2.o)
                0x00013930                __gtdf2
 *fill*         0x00013952        0x2 00
 .text          0x00013954       0x22 /opt/toolchains/sega/m68k-elf/lib/gcc/m68k-elf/4.6.2/libgcc.a(_gedf2.o)
                0x00013954                __gedf2
 *fill*         0x00013976        0x2 00
 .text          0x00013978       0x22 /opt/toolchains/sega/m68k-elf/lib/gcc/m68k-elf/4.6.2/libgcc.a(_ltdf2.o)
                0x00013978                __ltdf2
 *fill*         0x0001399a        0x2 00
 .text          0x0001399c       0x74 /opt/toolchains/sega/m68k-elf/lib/gcc/m68k-elf/4.6.2/libgcc.a(_muldi3.o)
                0x0001399c                __muldi3
 .text          0x00013a10      0x462 /opt/toolchains/sega/m68k-elf/lib/gcc/m68k-elf/4.6.2/libgcc.a(fpgnulib.o)
                0x00013a10                __unordsf2
                0x00013a5e                __unorddf2
                0x00013ada                __floatunsidf
                0x00013b46                __floatsidf
                0x00013be0                __floatunsisf
                0x00013bfa                __floatsisf
                0x00013c14                __extendsfdf2
                0x00013c94                __truncdfsf2
                0x00013dd2                __fixdfsi
                0x00013e58                __fixsfsi
 *fill*         0x00013e72        0x2 00
 .text          0x00013e74      0x7ae /opt/toolchains/sega/m68k-elf/lib/gcc/m68k-elf/4.6.2/libgcc.a(xfgnulib.o)
                0x00013e74                __unordxf2
                0x00013efe                __extenddfxf2
                0x00013fb8                __truncxfdf2
                0x00014088                __extendsfxf2
                0x000140cc                __truncxfsf2
                0x000140f4                __floatsixf
                0x0001413a                __floatunsixf
                0x00014180                __fixxfsi
                0x000141a8                __addxf3
                0x0001421e                __subxf3
                0x00014294                __mulxf3
                0x0001430a                __divxf3
                0x00014380                __negxf2
                0x000143d6                __cmpxf2
                0x0001442a                __eqxf2
                0x0001447e                __nexf2
                0x000144d2                __ltxf2
                0x00014526                __lexf2
                0x0001457a                __gtxf2
                0x000145ce                __gexf2
 *fill*         0x00014622        0x2 00
 .text          0x00014624       0x32 /opt/toolchains/sega/m68k-elf/m68k-elf/lib/libnosys.a(sbrk.o)
                0x00014624                sbrk
 *(.text.*)
 *(.gnu.linkonce.t.*)
                0x00014660                . = ALIGN (0x10)
 *fill*         0x00014656        0xa 00
                0x00014660                __INIT_SECTION__ = .
 *(.init)
                0x00014660        0x2 SHORT 0x4e75
                0x00014670                . = ALIGN (0x10)
 *fill*         0x00014662        0xe 00
                0x00014670                __FINI_SECTION__ = .
 *(.fini)
                0x00014670        0x2 SHORT 0x4e75
 *(.eh_frame_hdr)
 *(.eh_frame)
 *fill*         0x00014672        0x2 00
 .eh_frame      0x00014674      0x140 /opt/toolchains/sega/m68k-elf/lib/gcc/m68k-elf/4.6.2/libgcc.a(fpgnulib.o)
 .eh_frame      0x000147b4      0x2f0 /opt/toolchains/sega/m68k-elf/lib/gcc/m68k-elf/4.6.2/libgcc.a(xfgnulib.o)
                                0x308 (size before relaxing)
 *(.gcc_except_table)
 *(.jcr)
                0x00014ab0                . = ALIGN (0x10)
 *fill*         0x00014aa4        0xc 00
                0x00014ab0                __CTOR_LIST__ = .
                0x00014ab0                ___CTOR_LIST__ = .
                0x00014ab0        0x4 LONG 0x0 (((__CTOR_END__ - __CTOR_LIST__) / 0x4) - 0x2)
 *(SORT(.ctors.*))
 *(.ctors)
                0x00014ab4        0x4 LONG 0x0
                0x00014ab8                __CTOR_END__ = .
                0x00014ac0                . = ALIGN (0x10)
 *fill*         0x00014ab8        0x8 00
                0x00014ac0                __DTOR_LIST__ = .
                0x00014ac0                ___DTOR_LIST__ = .
                0x00014ac0        0x4 LONG 0x0 (((__DTOR_END__ - __DTOR_LIST__) / 0x4) - 0x2)
 *(SORT(.dtors.*))
 *(.dtors)
                0x00014ac4        0x4 LONG 0x0
                0x00014ac8                __DTOR_END__ = .
 *(.rdata)
 *(.rodata)
 .rodata        0x00014ac8       0x20 main.o
 .rodata        0x00014ae8      0x4a0 module.o
 .rodata        0x00014f88       0x20 /opt/toolchains/sega/m68k-elf/m68k-elf/lib/libc.a(lib_a-svfprintf.o)
 .rodata        0x00014fa8        0x4 /opt/toolchains/sega/m68k-elf/m68k-elf/lib/libc.a(lib_a-impure.o)
                0x00014fa8                _global_impure_ptr
 .rodata        0x00014fac      0x124 /opt/toolchains/sega/m68k-elf/m68k-elf/lib/libc.a(lib_a-mprec.o)
                0x00014fac                __mprec_tinytens
                0x00014fd4                __mprec_bigtens
                0x00014ffc                __mprec_tens
 .rodata        0x000150d0       0x20 /opt/toolchains/sega/m68k-elf/m68k-elf/lib/libc.a(lib_a-svfiprintf.o)
 *(.rodata.*)
 .rodata.str1.1
                0x000150f0      0x167 main.o
                                0x168 (size before relaxing)
 .rodata.str1.1
                0x00015257       0x3b /opt/toolchains/sega/m68k-elf/m68k-elf/lib/libc.a(lib_a-svfprintf.o)
 .rodata.str1.1
                0x00015292        0xd /opt/toolchains/sega/m68k-elf/m68k-elf/lib/libc.a(lib_a-dtoa.o)
                                  0xf (size before relaxing)
 .rodata.str1.1
                0x0001529f        0x2 /opt/toolchains/sega/m68k-elf/m68k-elf/lib/libc.a(lib_a-impure.o)
 .rodata.str1.1
                0x000152a1        0x6 /opt/toolchains/sega/m68k-elf/m68k-elf/lib/libc.a(lib_a-locale.o)
                                  0xb (size before relaxing)
 .rodata.str1.1
                0x00000000       0x29 /opt/toolchains/sega/m68k-elf/m68k-elf/lib/libc.a(lib_a-svfiprintf.o)
 *(.gnu.linkonce.r.*)
                0x000152b0                . = ALIGN (0x10)
 *fill*         0x000152a7        0x9 00
                0x000152b0                __text_end = .
                0x0000d2b0                __text_size = (__text_end - __text_start)

.data           0x000152b0      0x918
                0x000152b0                __data_start = .
 *(.data)
 .data          0x000152b0        0x4 crt0.o
 .data          0x000152b4        0x6 main.o
                0x000152b4                temp
                0x000152b8                gFilter
 *fill*         0x000152ba        0x2 00
 .data          0x000152bc        0x1 module.o
 *fill*         0x000152bd        0x3 00
 .data          0x000152c0        0x0 cdfh.o
 .data          0x000152c0        0xc hw_md.o
                0x000152c0                global_vars
 .data          0x000152cc       0x20 /opt/toolchains/sega/m68k-elf/lib/libpcm.a(pcm.o)
 .data          0x000152ec        0x6 /opt/toolchains/sega/m68k-elf/lib/libpcm.a(pcm-io.o)
 *fill*         0x000152f2        0x2 00
 .data          0x000152f4        0x0 /opt/toolchains/sega/m68k-elf/m68k-elf/lib/libc.a(lib_a-malloc.o)
 .data          0x000152f4      0x410 /opt/toolchains/sega/m68k-elf/m68k-elf/lib/libc.a(lib_a-mallocr.o)
                0x000152f4                __malloc_sbrk_base
                0x000152f8                __malloc_trim_threshold
                0x000152fc                __malloc_av_
 .data          0x00015704        0x0 /opt/toolchains/sega/m68k-elf/m68k-elf/lib/libc.a(lib_a-memcmp.o)
 .data          0x00015704        0x0 /opt/toolchains/sega/m68k-elf/m68k-elf/lib/libc.a(lib_a-memcpy.o)
 .data          0x00015704        0x0 /opt/toolchains/sega/m68k-elf/m68k-elf/lib/libc.a(lib_a-memset.o)
 .data          0x00015704        0x0 /opt/toolchains/sega/m68k-elf/m68k-elf/lib/libc.a(lib_a-mlock.o)
 .data          0x00015704        0x0 /opt/toolchains/sega/m68k-elf/m68k-elf/lib/libc.a(lib_a-rand.o)
 .data          0x00015704        0x0 /opt/toolchains/sega/m68k-elf/m68k-elf/lib/libc.a(lib_a-sbrkr.o)
 .data          0x00015704        0x0 /opt/toolchains/sega/m68k-elf/m68k-elf/lib/libc.a(lib_a-sprintf.o)
 .data          0x00015704        0x0 /opt/toolchains/sega/m68k-elf/m68k-elf/lib/libc.a(lib_a-strcat.o)
 .data          0x00015704        0x0 /opt/toolchains/sega/m68k-elf/m68k-elf/lib/libc.a(lib_a-strcpy.o)
 .data          0x00015704        0x0 /opt/toolchains/sega/m68k-elf/m68k-elf/lib/libc.a(lib_a-strlen.o)
 .data          0x00015704        0x0 /opt/toolchains/sega/m68k-elf/m68k-elf/lib/libc.a(lib_a-strncpy.o)
 .data          0x00015704        0x0 /opt/toolchains/sega/m68k-elf/m68k-elf/lib/libc.a(lib_a-svfprintf.o)
 .data          0x00015704        0x0 /opt/toolchains/sega/m68k-elf/m68k-elf/lib/libc.a(lib_a-dtoa.o)
 .data          0x00015704        0x0 /opt/toolchains/sega/m68k-elf/m68k-elf/lib/libc.a(lib_a-freer.o)
 .data          0x00015704      0x426 /opt/toolchains/sega/m68k-elf/m68k-elf/lib/libc.a(lib_a-impure.o)
                0x00015704                _impure_ptr
 *fill*         0x00015b2a        0x2 00
 .data          0x00015b2c       0x7a /opt/toolchains/sega/m68k-elf/m68k-elf/lib/libc.a(lib_a-locale.o)
                0x00015b2c                __mb_cur_max
 *fill*         0x00015ba6        0x2 00
 .data          0x00015ba8        0x0 /opt/toolchains/sega/m68k-elf/m68k-elf/lib/libc.a(lib_a-memchr.o)
 .data          0x00015ba8        0x0 /opt/toolchains/sega/m68k-elf/m68k-elf/lib/libc.a(lib_a-mprec.o)
 .data          0x00015ba8        0x0 /opt/toolchains/sega/m68k-elf/m68k-elf/lib/libc.a(lib_a-reent.o)
 .data          0x00015ba8        0x0 /opt/toolchains/sega/m68k-elf/m68k-elf/lib/libc.a(lib_a-s_fpclassify.o)
 .data          0x00015ba8        0x0 /opt/toolchains/sega/m68k-elf/m68k-elf/lib/libc.a(lib_a-strcmp.o)
 .data          0x00015ba8        0x0 /opt/toolchains/sega/m68k-elf/m68k-elf/lib/libc.a(lib_a-svfiprintf.o)
 .data          0x00015ba8        0x0 /opt/toolchains/sega/m68k-elf/m68k-elf/lib/libc.a(lib_a-callocr.o)
 .data          0x00015ba8        0x0 /opt/toolchains/sega/m68k-elf/m68k-elf/lib/libc.a(lib_a-memmove.o)
 .data          0x00015ba8        0x0 /opt/toolchains/sega/m68k-elf/m68k-elf/lib/libc.a(lib_a-reallocr.o)
 .data          0x00015ba8        0x0 /opt/toolchains/sega/m68k-elf/lib/gcc/m68k-elf/4.6.2/libgcc.a(_mulsi3.o)
 .data          0x00015ba8        0x0 /opt/toolchains/sega/m68k-elf/lib/gcc/m68k-elf/4.6.2/libgcc.a(_udivsi3.o)
 .data          0x00015ba8        0x0 /opt/toolchains/sega/m68k-elf/lib/gcc/m68k-elf/4.6.2/libgcc.a(_divsi3.o)
 .data          0x00015ba8        0x0 /opt/toolchains/sega/m68k-elf/lib/gcc/m68k-elf/4.6.2/libgcc.a(_umodsi3.o)
 .data          0x00015ba8        0x0 /opt/toolchains/sega/m68k-elf/lib/gcc/m68k-elf/4.6.2/libgcc.a(_modsi3.o)
 .data          0x00015ba8        0x0 /opt/toolchains/sega/m68k-elf/lib/gcc/m68k-elf/4.6.2/libgcc.a(_double.o)
 .data          0x00015ba8       0x1c /opt/toolchains/sega/m68k-elf/lib/gcc/m68k-elf/4.6.2/libgcc.a(_floatex.o)
                0x00015ba8                _fpCCR
 .data          0x00015bc4        0x0 /opt/toolchains/sega/m68k-elf/lib/gcc/m68k-elf/4.6.2/libgcc.a(_eqdf2.o)
 .data          0x00015bc4        0x0 /opt/toolchains/sega/m68k-elf/lib/gcc/m68k-elf/4.6.2/libgcc.a(_nedf2.o)
 .data          0x00015bc4        0x0 /opt/toolchains/sega/m68k-elf/lib/gcc/m68k-elf/4.6.2/libgcc.a(_gtdf2.o)
 .data          0x00015bc4        0x0 /opt/toolchains/sega/m68k-elf/lib/gcc/m68k-elf/4.6.2/libgcc.a(_gedf2.o)
 .data          0x00015bc4        0x0 /opt/toolchains/sega/m68k-elf/lib/gcc/m68k-elf/4.6.2/libgcc.a(_ltdf2.o)
 .data          0x00015bc4        0x0 /opt/toolchains/sega/m68k-elf/lib/gcc/m68k-elf/4.6.2/libgcc.a(_muldi3.o)
 .data          0x00015bc4        0x0 /opt/toolchains/sega/m68k-elf/lib/gcc/m68k-elf/4.6.2/libgcc.a(fpgnulib.o)
 .data          0x00015bc4        0x0 /opt/toolchains/sega/m68k-elf/lib/gcc/m68k-elf/4.6.2/libgcc.a(xfgnulib.o)
 .data          0x00015bc4        0x0 /opt/toolchains/sega/m68k-elf/m68k-elf/lib/libnosys.a(sbrk.o)
 *(.data.*)
 *(.gnu.linkonce.d.*)
 *(.lit8)
 *(.lit4)
 *(.sdata)
 *(.sdata.*)
 *(.gnu.linkonce.s.*)
                0x00015bc8                . = ALIGN (0x8)
 *fill*         0x00015bc4        0x4 00
                0x00015bc8                __data_end = .
                0x00000918                __data_size = (__data_end - __data_start)

.bss            0x00015bc8    0x100d0
                0x00015bc8                __bss_start = .
 *(.bss)
 .bss           0x00015bc8        0x0 crt0.o
 .bss           0x00015bc8        0x6 main.o
                0x00015bc8                gCurrent
                0x00015bca                gFirst
                0x00015bcc                gCount
 *fill*         0x00015bce        0x2 00
 .bss           0x00015bd0        0x7 module.o
 *fill*         0x00015bd7        0x1 00
 .bss           0x00015bd8        0x0 cdfh.o
 .bss           0x00015bd8        0x0 hw_md.o
 .bss           0x00015bd8        0x1 /opt/toolchains/sega/m68k-elf/lib/libpcm.a(pcm.o)
 *fill*         0x00015bd9        0x3 00
 .bss           0x00015bdc        0x0 /opt/toolchains/sega/m68k-elf/lib/libpcm.a(pcm-io.o)
 .bss           0x00015bdc        0x0 /opt/toolchains/sega/m68k-elf/m68k-elf/lib/libc.a(lib_a-malloc.o)
 .bss           0x00015bdc       0x34 /opt/toolchains/sega/m68k-elf/m68k-elf/lib/libc.a(lib_a-mallocr.o)
                0x00015bdc                __malloc_current_mallinfo
                0x00015c04                __malloc_max_total_mem
                0x00015c08                __malloc_max_sbrked_mem
                0x00015c0c                __malloc_top_pad
 .bss           0x00015c10        0x0 /opt/toolchains/sega/m68k-elf/m68k-elf/lib/libc.a(lib_a-memcmp.o)
 .bss           0x00015c10        0x0 /opt/toolchains/sega/m68k-elf/m68k-elf/lib/libc.a(lib_a-memcpy.o)
 .bss           0x00015c10        0x0 /opt/toolchains/sega/m68k-elf/m68k-elf/lib/libc.a(lib_a-memset.o)
 .bss           0x00015c10        0x0 /opt/toolchains/sega/m68k-elf/m68k-elf/lib/libc.a(lib_a-mlock.o)
 .bss           0x00015c10        0x0 /opt/toolchains/sega/m68k-elf/m68k-elf/lib/libc.a(lib_a-rand.o)
 .bss           0x00015c10        0x0 /opt/toolchains/sega/m68k-elf/m68k-elf/lib/libc.a(lib_a-sbrkr.o)
 .bss           0x00015c10        0x0 /opt/toolchains/sega/m68k-elf/m68k-elf/lib/libc.a(lib_a-sprintf.o)
 .bss           0x00015c10        0x0 /opt/toolchains/sega/m68k-elf/m68k-elf/lib/libc.a(lib_a-strcat.o)
 .bss           0x00015c10        0x0 /opt/toolchains/sega/m68k-elf/m68k-elf/lib/libc.a(lib_a-strcpy.o)
 .bss           0x00015c10        0x0 /opt/toolchains/sega/m68k-elf/m68k-elf/lib/libc.a(lib_a-strlen.o)
 .bss           0x00015c10        0x0 /opt/toolchains/sega/m68k-elf/m68k-elf/lib/libc.a(lib_a-strncpy.o)
 .bss           0x00015c10        0x0 /opt/toolchains/sega/m68k-elf/m68k-elf/lib/libc.a(lib_a-svfprintf.o)
 .bss           0x00015c10        0x0 /opt/toolchains/sega/m68k-elf/m68k-elf/lib/libc.a(lib_a-dtoa.o)
 .bss           0x00015c10        0x0 /opt/toolchains/sega/m68k-elf/m68k-elf/lib/libc.a(lib_a-freer.o)
 .bss           0x00015c10        0x0 /opt/toolchains/sega/m68k-elf/m68k-elf/lib/libc.a(lib_a-impure.o)
 .bss           0x00015c10        0xc /opt/toolchains/sega/m68k-elf/m68k-elf/lib/libc.a(lib_a-locale.o)
                0x00015c10                _PathLocale
                0x00015c14                __mlocale_changed
                0x00015c18                __nlocale_changed
 .bss           0x00015c1c        0x0 /opt/toolchains/sega/m68k-elf/m68k-elf/lib/libc.a(lib_a-memchr.o)
 .bss           0x00015c1c        0x0 /opt/toolchains/sega/m68k-elf/m68k-elf/lib/libc.a(lib_a-mprec.o)
 .bss           0x00015c1c        0x0 /opt/toolchains/sega/m68k-elf/m68k-elf/lib/libc.a(lib_a-reent.o)
 .bss           0x00015c1c        0x0 /opt/toolchains/sega/m68k-elf/m68k-elf/lib/libc.a(lib_a-s_fpclassify.o)
 .bss           0x00015c1c        0x0 /opt/toolchains/sega/m68k-elf/m68k-elf/lib/libc.a(lib_a-strcmp.o)
 .bss           0x00015c1c        0x0 /opt/toolchains/sega/m68k-elf/m68k-elf/lib/libc.a(lib_a-svfiprintf.o)
 .bss           0x00015c1c        0x0 /opt/toolchains/sega/m68k-elf/m68k-elf/lib/libc.a(lib_a-callocr.o)
 .bss           0x00015c1c        0x0 /opt/toolchains/sega/m68k-elf/m68k-elf/lib/libc.a(lib_a-memmove.o)
 .bss           0x00015c1c        0x0 /opt/toolchains/sega/m68k-elf/m68k-elf/lib/libc.a(lib_a-reallocr.o)
 .bss           0x00015c1c        0x0 /opt/toolchains/sega/m68k-elf/lib/gcc/m68k-elf/4.6.2/libgcc.a(_mulsi3.o)
 .bss           0x00015c1c        0x0 /opt/toolchains/sega/m68k-elf/lib/gcc/m68k-elf/4.6.2/libgcc.a(_udivsi3.o)
 .bss           0x00015c1c        0x0 /opt/toolchains/sega/m68k-elf/lib/gcc/m68k-elf/4.6.2/libgcc.a(_divsi3.o)
 .bss           0x00015c1c        0x0 /opt/toolchains/sega/m68k-elf/lib/gcc/m68k-elf/4.6.2/libgcc.a(_umodsi3.o)
 .bss           0x00015c1c        0x0 /opt/toolchains/sega/m68k-elf/lib/gcc/m68k-elf/4.6.2/libgcc.a(_modsi3.o)
 .bss           0x00015c1c        0x0 /opt/toolchains/sega/m68k-elf/lib/gcc/m68k-elf/4.6.2/libgcc.a(_double.o)
 .bss           0x00015c1c        0x0 /opt/toolchains/sega/m68k-elf/lib/gcc/m68k-elf/4.6.2/libgcc.a(_floatex.o)
 .bss           0x00015c1c        0x0 /opt/toolchains/sega/m68k-elf/lib/gcc/m68k-elf/4.6.2/libgcc.a(_eqdf2.o)
 .bss           0x00015c1c        0x0 /opt/toolchains/sega/m68k-elf/lib/gcc/m68k-elf/4.6.2/libgcc.a(_nedf2.o)
 .bss           0x00015c1c        0x0 /opt/toolchains/sega/m68k-elf/lib/gcc/m68k-elf/4.6.2/libgcc.a(_gtdf2.o)
 .bss           0x00015c1c        0x0 /opt/toolchains/sega/m68k-elf/lib/gcc/m68k-elf/4.6.2/libgcc.a(_gedf2.o)
 .bss           0x00015c1c        0x0 /opt/toolchains/sega/m68k-elf/lib/gcc/m68k-elf/4.6.2/libgcc.a(_ltdf2.o)
 .bss           0x00015c1c        0x0 /opt/toolchains/sega/m68k-elf/lib/gcc/m68k-elf/4.6.2/libgcc.a(_muldi3.o)
 .bss           0x00015c1c        0x0 /opt/toolchains/sega/m68k-elf/lib/gcc/m68k-elf/4.6.2/libgcc.a(fpgnulib.o)
 .bss           0x00015c1c        0x0 /opt/toolchains/sega/m68k-elf/lib/gcc/m68k-elf/4.6.2/libgcc.a(xfgnulib.o)
 .bss           0x00015c1c        0x4 /opt/toolchains/sega/m68k-elf/m68k-elf/lib/libnosys.a(sbrk.o)
 *(.bss.*)
 *(.gnu.linkonce.b.*)
 *(.sbss)
 *(.sbss.*)
 *(.gnu.linkonce.sb.*)
 *(.scommon)
 *(COMMON)
 COMMON         0x00015c20    0x10000 main.o
                0x00015c20                gDirTable
 COMMON         0x00025c20       0x70 module.o
                0x00025c20                voices
 COMMON         0x00025c90        0x4 /opt/toolchains/sega/m68k-elf/m68k-elf/lib/libc.a(lib_a-reent.o)
                0x00025c90                errno
                0x00025c98                . = ALIGN (0x8)
 *fill*         0x00025c94        0x4 00
                0x00025c98                end = .
                0x00025c98                _end = end
                0x00025c98                __end = _end
                0x00025c98                __bss_end = .
                0x000100d0                __bss_size = (__bss_end - __bss_start)
OUTPUT(CDModPlayer.elf elf32-m68k)

.comment        0x00000000       0x11
 .comment       0x00000000       0x11 main.o
                                 0x12 (size before relaxing)
 .comment       0x00000000       0x12 module.o
 .comment       0x00000000       0x12 cdfh.o
 .comment       0x00000000       0x12 /opt/toolchains/sega/m68k-elf/lib/libpcm.a(pcm.o)
 .comment       0x00000000       0x12 /opt/toolchains/sega/m68k-elf/m68k-elf/lib/libc.a(lib_a-malloc.o)
 .comment       0x00000000       0x12 /opt/toolchains/sega/m68k-elf/m68k-elf/lib/libc.a(lib_a-mallocr.o)
 .comment       0x00000000       0x12 /opt/toolchains/sega/m68k-elf/m68k-elf/lib/libc.a(lib_a-memcmp.o)
 .comment       0x00000000       0x12 /opt/toolchains/sega/m68k-elf/m68k-elf/lib/libc.a(lib_a-mlock.o)
 .comment       0x00000000       0x12 /opt/toolchains/sega/m68k-elf/m68k-elf/lib/libc.a(lib_a-rand.o)
 .comment       0x00000000       0x12 /opt/toolchains/sega/m68k-elf/m68k-elf/lib/libc.a(lib_a-sbrkr.o)
 .comment       0x00000000       0x12 /opt/toolchains/sega/m68k-elf/m68k-elf/lib/libc.a(lib_a-sprintf.o)
 .comment       0x00000000       0x12 /opt/toolchains/sega/m68k-elf/m68k-elf/lib/libc.a(lib_a-strcat.o)
 .comment       0x00000000       0x12 /opt/toolchains/sega/m68k-elf/m68k-elf/lib/libc.a(lib_a-strcpy.o)
 .comment       0x00000000       0x12 /opt/toolchains/sega/m68k-elf/m68k-elf/lib/libc.a(lib_a-strlen.o)
 .comment       0x00000000       0x12 /opt/toolchains/sega/m68k-elf/m68k-elf/lib/libc.a(lib_a-strncpy.o)
 .comment       0x00000000       0x12 /opt/toolchains/sega/m68k-elf/m68k-elf/lib/libc.a(lib_a-svfprintf.o)
 .comment       0x00000000       0x12 /opt/toolchains/sega/m68k-elf/m68k-elf/lib/libc.a(lib_a-dtoa.o)
 .comment       0x00000000       0x12 /opt/toolchains/sega/m68k-elf/m68k-elf/lib/libc.a(lib_a-freer.o)
 .comment       0x00000000       0x12 /opt/toolchains/sega/m68k-elf/m68k-elf/lib/libc.a(lib_a-impure.o)
 .comment       0x00000000       0x12 /opt/toolchains/sega/m68k-elf/m68k-elf/lib/libc.a(lib_a-locale.o)
 .comment       0x00000000       0x12 /opt/toolchains/sega/m68k-elf/m68k-elf/lib/libc.a(lib_a-memchr.o)
 .comment       0x00000000       0x12 /opt/toolchains/sega/m68k-elf/m68k-elf/lib/libc.a(lib_a-mprec.o)
 .comment       0x00000000       0x12 /opt/toolchains/sega/m68k-elf/m68k-elf/lib/libc.a(lib_a-reent.o)
 .comment       0x00000000       0x12 /opt/toolchains/sega/m68k-elf/m68k-elf/lib/libc.a(lib_a-s_fpclassify.o)
 .comment       0x00000000       0x12 /opt/toolchains/sega/m68k-elf/m68k-elf/lib/libc.a(lib_a-strcmp.o)
 .comment       0x00000000       0x12 /opt/toolchains/sega/m68k-elf/m68k-elf/lib/libc.a(lib_a-svfiprintf.o)
 .comment       0x00000000       0x12 /opt/toolchains/sega/m68k-elf/m68k-elf/lib/libc.a(lib_a-callocr.o)
 .comment       0x00000000       0x12 /opt/toolchains/sega/m68k-elf/m68k-elf/lib/libc.a(lib_a-memmove.o)
 .comment       0x00000000       0x12 /opt/toolchains/sega/m68k-elf/m68k-elf/lib/libc.a(lib_a-reallocr.o)
 .comment       0x00000000       0x12 /opt/toolchains/sega/m68k-elf/lib/gcc/m68k-elf/4.6.2/libgcc.a(_muldi3.o)
 .comment       0x00000000       0x12 /opt/toolchains/sega/m68k-elf/lib/gcc/m68k-elf/4.6.2/libgcc.a(fpgnulib.o)
 .comment       0x00000000       0x12 /opt/toolchains/sega/m68k-elf/lib/gcc/m68k-elf/4.6.2/libgcc.a(xfgnulib.o)
 .comment       0x00000000       0x12 /opt/toolchains/sega/m68k-elf/m68k-elf/lib/libnosys.a(sbrk.o)

.debug_info     0x00000000     0xdfd8
 .debug_info    0x00000000      0x9a4 /opt/toolchains/sega/m68k-elf/m68k-elf/lib/libc.a(lib_a-malloc.o)
 .debug_info    0x000009a4      0xd68 /opt/toolchains/sega/m68k-elf/m68k-elf/lib/libc.a(lib_a-mallocr.o)
 .debug_info    0x0000170c      0x10e /opt/toolchains/sega/m68k-elf/m68k-elf/lib/libc.a(lib_a-memcmp.o)
 .debug_info    0x0000181a       0xca /opt/toolchains/sega/m68k-elf/m68k-elf/lib/libc.a(lib_a-memcpy.o)
 .debug_info    0x000018e4       0xca /opt/toolchains/sega/m68k-elf/m68k-elf/lib/libc.a(lib_a-memset.o)
 .debug_info    0x000019ae      0x983 /opt/toolchains/sega/m68k-elf/m68k-elf/lib/libc.a(lib_a-mlock.o)
 .debug_info    0x00002331      0x986 /opt/toolchains/sega/m68k-elf/m68k-elf/lib/libc.a(lib_a-rand.o)
 .debug_info    0x00002cb7      0x9a9 /opt/toolchains/sega/m68k-elf/m68k-elf/lib/libc.a(lib_a-sbrkr.o)
 .debug_info    0x00003660      0xa4c /opt/toolchains/sega/m68k-elf/m68k-elf/lib/libc.a(lib_a-sprintf.o)
 .debug_info    0x000040ac       0xe4 /opt/toolchains/sega/m68k-elf/m68k-elf/lib/libc.a(lib_a-strcat.o)
 .debug_info    0x00004190       0xd5 /opt/toolchains/sega/m68k-elf/m68k-elf/lib/libc.a(lib_a-strcpy.o)
 .debug_info    0x00004265       0xcc /opt/toolchains/sega/m68k-elf/m68k-elf/lib/libc.a(lib_a-strlen.o)
 .debug_info    0x00004331      0x125 /opt/toolchains/sega/m68k-elf/m68k-elf/lib/libc.a(lib_a-strncpy.o)
 .debug_info    0x00004456      0xffb /opt/toolchains/sega/m68k-elf/m68k-elf/lib/libc.a(lib_a-svfprintf.o)
 .debug_info    0x00005451      0xdc6 /opt/toolchains/sega/m68k-elf/m68k-elf/lib/libc.a(lib_a-dtoa.o)
 .debug_info    0x00006217      0xc3b /opt/toolchains/sega/m68k-elf/m68k-elf/lib/libc.a(lib_a-freer.o)
 .debug_info    0x00006e52      0x965 /opt/toolchains/sega/m68k-elf/m68k-elf/lib/libc.a(lib_a-impure.o)
 .debug_info    0x000077b7      0xc96 /opt/toolchains/sega/m68k-elf/m68k-elf/lib/libc.a(lib_a-locale.o)
 .debug_info    0x0000844d      0x122 /opt/toolchains/sega/m68k-elf/m68k-elf/lib/libc.a(lib_a-memchr.o)
 .debug_info    0x0000856f     0x14d7 /opt/toolchains/sega/m68k-elf/m68k-elf/lib/libc.a(lib_a-mprec.o)
 .debug_info    0x00009a46      0xa60 /opt/toolchains/sega/m68k-elf/m68k-elf/lib/libc.a(lib_a-reent.o)
 .debug_info    0x0000a4a6      0x13f /opt/toolchains/sega/m68k-elf/m68k-elf/lib/libc.a(lib_a-s_fpclassify.o)
 .debug_info    0x0000a5e5       0xda /opt/toolchains/sega/m68k-elf/m68k-elf/lib/libc.a(lib_a-strcmp.o)
 .debug_info    0x0000a6bf      0xd7b /opt/toolchains/sega/m68k-elf/m68k-elf/lib/libc.a(lib_a-svfiprintf.o)
 .debug_info    0x0000b43a      0xa4b /opt/toolchains/sega/m68k-elf/m68k-elf/lib/libc.a(lib_a-callocr.o)
 .debug_info    0x0000be85      0x12e /opt/toolchains/sega/m68k-elf/m68k-elf/lib/libc.a(lib_a-memmove.o)
 .debug_info    0x0000bfb3      0xc00 /opt/toolchains/sega/m68k-elf/m68k-elf/lib/libc.a(lib_a-reallocr.o)
 .debug_info    0x0000cbb3       0xab /opt/toolchains/sega/m68k-elf/lib/gcc/m68k-elf/4.6.2/libgcc.a(_mulsi3.o)
 .debug_info    0x0000cc5e       0xab /opt/toolchains/sega/m68k-elf/lib/gcc/m68k-elf/4.6.2/libgcc.a(_udivsi3.o)
 .debug_info    0x0000cd09       0xab /opt/toolchains/sega/m68k-elf/lib/gcc/m68k-elf/4.6.2/libgcc.a(_divsi3.o)
 .debug_info    0x0000cdb4       0xab /opt/toolchains/sega/m68k-elf/lib/gcc/m68k-elf/4.6.2/libgcc.a(_umodsi3.o)
 .debug_info    0x0000ce5f       0xab /opt/toolchains/sega/m68k-elf/lib/gcc/m68k-elf/4.6.2/libgcc.a(_modsi3.o)
 .debug_info    0x0000cf0a       0xab /opt/toolchains/sega/m68k-elf/lib/gcc/m68k-elf/4.6.2/libgcc.a(_double.o)
 .debug_info    0x0000cfb5       0xab /opt/toolchains/sega/m68k-elf/lib/gcc/m68k-elf/4.6.2/libgcc.a(_floatex.o)
 .debug_info    0x0000d060       0xab /opt/toolchains/sega/m68k-elf/lib/gcc/m68k-elf/4.6.2/libgcc.a(_eqdf2.o)
 .debug_info    0x0000d10b       0xab /opt/toolchains/sega/m68k-elf/lib/gcc/m68k-elf/4.6.2/libgcc.a(_nedf2.o)
 .debug_info    0x0000d1b6       0xab /opt/toolchains/sega/m68k-elf/lib/gcc/m68k-elf/4.6.2/libgcc.a(_gtdf2.o)
 .debug_info    0x0000d261       0xab /opt/toolchains/sega/m68k-elf/lib/gcc/m68k-elf/4.6.2/libgcc.a(_gedf2.o)
 .debug_info    0x0000d30c       0xab /opt/toolchains/sega/m68k-elf/lib/gcc/m68k-elf/4.6.2/libgcc.a(_ltdf2.o)
 .debug_info    0x0000d3b7      0x182 /opt/toolchains/sega/m68k-elf/lib/gcc/m68k-elf/4.6.2/libgcc.a(_muldi3.o)
 .debug_info    0x0000d539      0x3db /opt/toolchains/sega/m68k-elf/lib/gcc/m68k-elf/4.6.2/libgcc.a(fpgnulib.o)
 .debug_info    0x0000d914      0x623 /opt/toolchains/sega/m68k-elf/lib/gcc/m68k-elf/4.6.2/libgcc.a(xfgnulib.o)
 .debug_info    0x0000df37       0xa1 /opt/toolchains/sega/m68k-elf/m68k-elf/lib/libnosys.a(sbrk.o)

.debug_abbrev   0x00000000     0x29e3
 .debug_abbrev  0x00000000      0x196 /opt/toolchains/sega/m68k-elf/m68k-elf/lib/libc.a(lib_a-malloc.o)
 .debug_abbrev  0x00000196      0x233 /opt/toolchains/sega/m68k-elf/m68k-elf/lib/libc.a(lib_a-mallocr.o)
 .debug_abbrev  0x000003c9       0x8b /opt/toolchains/sega/m68k-elf/m68k-elf/lib/libc.a(lib_a-memcmp.o)
 .debug_abbrev  0x00000454       0x14 /opt/toolchains/sega/m68k-elf/m68k-elf/lib/libc.a(lib_a-memcpy.o)
 .debug_abbrev  0x00000468       0x14 /opt/toolchains/sega/m68k-elf/m68k-elf/lib/libc.a(lib_a-memset.o)
 .debug_abbrev  0x0000047c      0x179 /opt/toolchains/sega/m68k-elf/m68k-elf/lib/libc.a(lib_a-mlock.o)
 .debug_abbrev  0x000005f5      0x194 /opt/toolchains/sega/m68k-elf/m68k-elf/lib/libc.a(lib_a-rand.o)
 .debug_abbrev  0x00000789      0x1b0 /opt/toolchains/sega/m68k-elf/m68k-elf/lib/libc.a(lib_a-sbrkr.o)
 .debug_abbrev  0x00000939      0x1b5 /opt/toolchains/sega/m68k-elf/m68k-elf/lib/libc.a(lib_a-sprintf.o)
 .debug_abbrev  0x00000aee       0x96 /opt/toolchains/sega/m68k-elf/m68k-elf/lib/libc.a(lib_a-strcat.o)
 .debug_abbrev  0x00000b84       0x7e /opt/toolchains/sega/m68k-elf/m68k-elf/lib/libc.a(lib_a-strcpy.o)
 .debug_abbrev  0x00000c02       0x7c /opt/toolchains/sega/m68k-elf/m68k-elf/lib/libc.a(lib_a-strlen.o)
 .debug_abbrev  0x00000c7e       0x9c /opt/toolchains/sega/m68k-elf/m68k-elf/lib/libc.a(lib_a-strncpy.o)
 .debug_abbrev  0x00000d1a      0x2f5 /opt/toolchains/sega/m68k-elf/m68k-elf/lib/libc.a(lib_a-svfprintf.o)
 .debug_abbrev  0x0000100f      0x229 /opt/toolchains/sega/m68k-elf/m68k-elf/lib/libc.a(lib_a-dtoa.o)
 .debug_abbrev  0x00001238      0x1ea /opt/toolchains/sega/m68k-elf/m68k-elf/lib/libc.a(lib_a-freer.o)
 .debug_abbrev  0x00001422      0x166 /opt/toolchains/sega/m68k-elf/m68k-elf/lib/libc.a(lib_a-impure.o)
 .debug_abbrev  0x00001588      0x245 /opt/toolchains/sega/m68k-elf/m68k-elf/lib/libc.a(lib_a-locale.o)
 .debug_abbrev  0x000017cd       0xd5 /opt/toolchains/sega/m68k-elf/m68k-elf/lib/libc.a(lib_a-memchr.o)
 .debug_abbrev  0x000018a2      0x2fa /opt/toolchains/sega/m68k-elf/m68k-elf/lib/libc.a(lib_a-mprec.o)
 .debug_abbrev  0x00001b9c      0x1f5 /opt/toolchains/sega/m68k-elf/m68k-elf/lib/libc.a(lib_a-reent.o)
 .debug_abbrev  0x00001d91       0xc5 /opt/toolchains/sega/m68k-elf/m68k-elf/lib/libc.a(lib_a-s_fpclassify.o)
 .debug_abbrev  0x00001e56       0x71 /opt/toolchains/sega/m68k-elf/m68k-elf/lib/libc.a(lib_a-strcmp.o)
 .debug_abbrev  0x00001ec7      0x26d /opt/toolchains/sega/m68k-elf/m68k-elf/lib/libc.a(lib_a-svfiprintf.o)
 .debug_abbrev  0x00002134      0x1c0 /opt/toolchains/sega/m68k-elf/m68k-elf/lib/libc.a(lib_a-callocr.o)
 .debug_abbrev  0x000022f4       0xa8 /opt/toolchains/sega/m68k-elf/m68k-elf/lib/libc.a(lib_a-memmove.o)
 .debug_abbrev  0x0000239c      0x1d2 /opt/toolchains/sega/m68k-elf/m68k-elf/lib/libc.a(lib_a-reallocr.o)
 .debug_abbrev  0x0000256e       0x14 /opt/toolchains/sega/m68k-elf/lib/gcc/m68k-elf/4.6.2/libgcc.a(_mulsi3.o)
 .debug_abbrev  0x00002582       0x14 /opt/toolchains/sega/m68k-elf/lib/gcc/m68k-elf/4.6.2/libgcc.a(_udivsi3.o)
 .debug_abbrev  0x00002596       0x14 /opt/toolchains/sega/m68k-elf/lib/gcc/m68k-elf/4.6.2/libgcc.a(_divsi3.o)
 .debug_abbrev  0x000025aa       0x14 /opt/toolchains/sega/m68k-elf/lib/gcc/m68k-elf/4.6.2/libgcc.a(_umodsi3.o)
 .debug_abbrev  0x000025be       0x14 /opt/toolchains/sega/m68k-elf/lib/gcc/m68k-elf/4.6.2/libgcc.a(_modsi3.o)
 .debug_abbrev  0x000025d2       0x14 /opt/toolchains/sega/m68k-elf/lib/gcc/m68k-elf/4.6.2/libgcc.a(_double.o)
 .debug_abbrev  0x000025e6       0x14 /opt/toolchains/sega/m68k-elf/lib/gcc/m68k-elf/4.6.2/libgcc.a(_floatex.o)
 .debug_abbrev  0x000025fa       0x14 /opt/toolchains/sega/m68k-elf/lib/gcc/m68k-elf/4.6.2/libgcc.a(_eqdf2.o)
 .debug_abbrev  0x0000260e       0x14 /opt/toolchains/sega/m68k-elf/lib/gcc/m68k-elf/4.6.2/libgcc.a(_nedf2.o)
 .debug_abbrev  0x00002622       0x14 /opt/toolchains/sega/m68k-elf/lib/gcc/m68k-elf/4.6.2/libgcc.a(_gtdf2.o)
 .debug_abbrev  0x00002636       0x14 /opt/toolchains/sega/m68k-elf/lib/gcc/m68k-elf/4.6.2/libgcc.a(_gedf2.o)
 .debug_abbrev  0x0000264a       0x14 /opt/toolchains/sega/m68k-elf/lib/gcc/m68k-elf/4.6.2/libgcc.a(_ltdf2.o)
 .debug_abbrev  0x0000265e       0xd0 /opt/toolchains/sega/m68k-elf/lib/gcc/m68k-elf/4.6.2/libgcc.a(_muldi3.o)
 .debug_abbrev  0x0000272e      0x144 /opt/toolchains/sega/m68k-elf/lib/gcc/m68k-elf/4.6.2/libgcc.a(fpgnulib.o)
 .debug_abbrev  0x00002872       0xe2 /opt/toolchains/sega/m68k-elf/lib/gcc/m68k-elf/4.6.2/libgcc.a(xfgnulib.o)
 .debug_abbrev  0x00002954       0x8f /opt/toolchains/sega/m68k-elf/m68k-elf/lib/libnosys.a(sbrk.o)

.debug_loc      0x00000000     0xa941
 .debug_loc     0x00000000       0x40 /opt/toolchains/sega/m68k-elf/m68k-elf/lib/libc.a(lib_a-malloc.o)
 .debug_loc     0x00000040      0xa7e /opt/toolchains/sega/m68k-elf/m68k-elf/lib/libc.a(lib_a-mallocr.o)
 .debug_loc     0x00000abe       0xe0 /opt/toolchains/sega/m68k-elf/m68k-elf/lib/libc.a(lib_a-memcmp.o)
 .debug_loc     0x00000b9e       0x40 /opt/toolchains/sega/m68k-elf/m68k-elf/lib/libc.a(lib_a-mlock.o)
 .debug_loc     0x00000bde       0x40 /opt/toolchains/sega/m68k-elf/m68k-elf/lib/libc.a(lib_a-rand.o)
 .debug_loc     0x00000c1e       0x20 /opt/toolchains/sega/m68k-elf/m68k-elf/lib/libc.a(lib_a-sbrkr.o)
 .debug_loc     0x00000c3e       0x40 /opt/toolchains/sega/m68k-elf/m68k-elf/lib/libc.a(lib_a-sprintf.o)
 .debug_loc     0x00000c7e       0x96 /opt/toolchains/sega/m68k-elf/m68k-elf/lib/libc.a(lib_a-strcat.o)
 .debug_loc     0x00000d14       0x4a /opt/toolchains/sega/m68k-elf/m68k-elf/lib/libc.a(lib_a-strcpy.o)
 .debug_loc     0x00000d5e       0x54 /opt/toolchains/sega/m68k-elf/m68k-elf/lib/libc.a(lib_a-strlen.o)
 .debug_loc     0x00000db2       0xf5 /opt/toolchains/sega/m68k-elf/m68k-elf/lib/libc.a(lib_a-strncpy.o)
 .debug_loc     0x00000ea7     0x277e /opt/toolchains/sega/m68k-elf/m68k-elf/lib/libc.a(lib_a-svfprintf.o)
 .debug_loc     0x00003625     0x1f6d /opt/toolchains/sega/m68k-elf/m68k-elf/lib/libc.a(lib_a-dtoa.o)
 .debug_loc     0x00005592      0x480 /opt/toolchains/sega/m68k-elf/m68k-elf/lib/libc.a(lib_a-freer.o)
 .debug_loc     0x00005a12      0x100 /opt/toolchains/sega/m68k-elf/m68k-elf/lib/libc.a(lib_a-locale.o)
 .debug_loc     0x00005b12      0x11e /opt/toolchains/sega/m68k-elf/m68k-elf/lib/libc.a(lib_a-memchr.o)
 .debug_loc     0x00005c30     0x178f /opt/toolchains/sega/m68k-elf/m68k-elf/lib/libc.a(lib_a-mprec.o)
 .debug_loc     0x000073bf      0x1f9 /opt/toolchains/sega/m68k-elf/m68k-elf/lib/libc.a(lib_a-reent.o)
 .debug_loc     0x000075b8       0x20 /opt/toolchains/sega/m68k-elf/m68k-elf/lib/libc.a(lib_a-s_fpclassify.o)
 .debug_loc     0x000075d8       0xf4 /opt/toolchains/sega/m68k-elf/m68k-elf/lib/libc.a(lib_a-strcmp.o)
 .debug_loc     0x000076cc     0x1304 /opt/toolchains/sega/m68k-elf/m68k-elf/lib/libc.a(lib_a-svfiprintf.o)
 .debug_loc     0x000089d0      0x222 /opt/toolchains/sega/m68k-elf/m68k-elf/lib/libc.a(lib_a-callocr.o)
 .debug_loc     0x00008bf2      0x19d /opt/toolchains/sega/m68k-elf/m68k-elf/lib/libc.a(lib_a-memmove.o)
 .debug_loc     0x00008d8f     0x1194 /opt/toolchains/sega/m68k-elf/m68k-elf/lib/libc.a(lib_a-reallocr.o)
 .debug_loc     0x00009f23       0x20 /opt/toolchains/sega/m68k-elf/lib/gcc/m68k-elf/4.6.2/libgcc.a(_muldi3.o)
 .debug_loc     0x00009f43      0x6c5 /opt/toolchains/sega/m68k-elf/lib/gcc/m68k-elf/4.6.2/libgcc.a(fpgnulib.o)
 .debug_loc     0x0000a608      0x2f7 /opt/toolchains/sega/m68k-elf/lib/gcc/m68k-elf/4.6.2/libgcc.a(xfgnulib.o)
 .debug_loc     0x0000a8ff       0x42 /opt/toolchains/sega/m68k-elf/m68k-elf/lib/libnosys.a(sbrk.o)

.debug_aranges  0x00000000      0x540
 .debug_aranges
                0x00000000       0x20 /opt/toolchains/sega/m68k-elf/m68k-elf/lib/libc.a(lib_a-malloc.o)
 .debug_aranges
                0x00000020       0x20 /opt/toolchains/sega/m68k-elf/m68k-elf/lib/libc.a(lib_a-mallocr.o)
 .debug_aranges
                0x00000040       0x20 /opt/toolchains/sega/m68k-elf/m68k-elf/lib/libc.a(lib_a-memcmp.o)
 .debug_aranges
                0x00000060       0x20 /opt/toolchains/sega/m68k-elf/m68k-elf/lib/libc.a(lib_a-memcpy.o)
 .debug_aranges
                0x00000080       0x20 /opt/toolchains/sega/m68k-elf/m68k-elf/lib/libc.a(lib_a-memset.o)
 .debug_aranges
                0x000000a0       0x20 /opt/toolchains/sega/m68k-elf/m68k-elf/lib/libc.a(lib_a-mlock.o)
 .debug_aranges
                0x000000c0       0x20 /opt/toolchains/sega/m68k-elf/m68k-elf/lib/libc.a(lib_a-rand.o)
 .debug_aranges
                0x000000e0       0x20 /opt/toolchains/sega/m68k-elf/m68k-elf/lib/libc.a(lib_a-sbrkr.o)
 .debug_aranges
                0x00000100       0x20 /opt/toolchains/sega/m68k-elf/m68k-elf/lib/libc.a(lib_a-sprintf.o)
 .debug_aranges
                0x00000120       0x20 /opt/toolchains/sega/m68k-elf/m68k-elf/lib/libc.a(lib_a-strcat.o)
 .debug_aranges
                0x00000140       0x20 /opt/toolchains/sega/m68k-elf/m68k-elf/lib/libc.a(lib_a-strcpy.o)
 .debug_aranges
                0x00000160       0x20 /opt/toolchains/sega/m68k-elf/m68k-elf/lib/libc.a(lib_a-strlen.o)
 .debug_aranges
                0x00000180       0x20 /opt/toolchains/sega/m68k-elf/m68k-elf/lib/libc.a(lib_a-strncpy.o)
 .debug_aranges
                0x000001a0       0x20 /opt/toolchains/sega/m68k-elf/m68k-elf/lib/libc.a(lib_a-svfprintf.o)
 .debug_aranges
                0x000001c0       0x20 /opt/toolchains/sega/m68k-elf/m68k-elf/lib/libc.a(lib_a-dtoa.o)
 .debug_aranges
                0x000001e0       0x20 /opt/toolchains/sega/m68k-elf/m68k-elf/lib/libc.a(lib_a-freer.o)
 .debug_aranges
                0x00000200       0x20 /opt/toolchains/sega/m68k-elf/m68k-elf/lib/libc.a(lib_a-locale.o)
 .debug_aranges
                0x00000220       0x20 /opt/toolchains/sega/m68k-elf/m68k-elf/lib/libc.a(lib_a-memchr.o)
 .debug_aranges
                0x00000240       0x20 /opt/toolchains/sega/m68k-elf/m68k-elf/lib/libc.a(lib_a-mprec.o)
 .debug_aranges
                0x00000260       0x20 /opt/toolchains/sega/m68k-elf/m68k-elf/lib/libc.a(lib_a-reent.o)
 .debug_aranges
                0x00000280       0x20 /opt/toolchains/sega/m68k-elf/m68k-elf/lib/libc.a(lib_a-s_fpclassify.o)
 .debug_aranges
                0x000002a0       0x20 /opt/toolchains/sega/m68k-elf/m68k-elf/lib/libc.a(lib_a-strcmp.o)
 .debug_aranges
                0x000002c0       0x20 /opt/toolchains/sega/m68k-elf/m68k-elf/lib/libc.a(lib_a-svfiprintf.o)
 .debug_aranges
                0x000002e0       0x20 /opt/toolchains/sega/m68k-elf/m68k-elf/lib/libc.a(lib_a-callocr.o)
 .debug_aranges
                0x00000300       0x20 /opt/toolchains/sega/m68k-elf/m68k-elf/lib/libc.a(lib_a-memmove.o)
 .debug_aranges
                0x00000320       0x20 /opt/toolchains/sega/m68k-elf/m68k-elf/lib/libc.a(lib_a-reallocr.o)
 .debug_aranges
                0x00000340       0x20 /opt/toolchains/sega/m68k-elf/lib/gcc/m68k-elf/4.6.2/libgcc.a(_mulsi3.o)
 .debug_aranges
                0x00000360       0x20 /opt/toolchains/sega/m68k-elf/lib/gcc/m68k-elf/4.6.2/libgcc.a(_udivsi3.o)
 .debug_aranges
                0x00000380       0x20 /opt/toolchains/sega/m68k-elf/lib/gcc/m68k-elf/4.6.2/libgcc.a(_divsi3.o)
 .debug_aranges
                0x000003a0       0x20 /opt/toolchains/sega/m68k-elf/lib/gcc/m68k-elf/4.6.2/libgcc.a(_umodsi3.o)
 .debug_aranges
                0x000003c0       0x20 /opt/toolchains/sega/m68k-elf/lib/gcc/m68k-elf/4.6.2/libgcc.a(_modsi3.o)
 .debug_aranges
                0x000003e0       0x20 /opt/toolchains/sega/m68k-elf/lib/gcc/m68k-elf/4.6.2/libgcc.a(_double.o)
 .debug_aranges
                0x00000400       0x20 /opt/toolchains/sega/m68k-elf/lib/gcc/m68k-elf/4.6.2/libgcc.a(_floatex.o)
 .debug_aranges
                0x00000420       0x20 /opt/toolchains/sega/m68k-elf/lib/gcc/m68k-elf/4.6.2/libgcc.a(_eqdf2.o)
 .debug_aranges
                0x00000440       0x20 /opt/toolchains/sega/m68k-elf/lib/gcc/m68k-elf/4.6.2/libgcc.a(_nedf2.o)
 .debug_aranges
                0x00000460       0x20 /opt/toolchains/sega/m68k-elf/lib/gcc/m68k-elf/4.6.2/libgcc.a(_gtdf2.o)
 .debug_aranges
                0x00000480       0x20 /opt/toolchains/sega/m68k-elf/lib/gcc/m68k-elf/4.6.2/libgcc.a(_gedf2.o)
 .debug_aranges
                0x000004a0       0x20 /opt/toolchains/sega/m68k-elf/lib/gcc/m68k-elf/4.6.2/libgcc.a(_ltdf2.o)
 .debug_aranges
                0x000004c0       0x20 /opt/toolchains/sega/m68k-elf/lib/gcc/m68k-elf/4.6.2/libgcc.a(_muldi3.o)
 .debug_aranges
                0x000004e0       0x20 /opt/toolchains/sega/m68k-elf/lib/gcc/m68k-elf/4.6.2/libgcc.a(fpgnulib.o)
 .debug_aranges
                0x00000500       0x20 /opt/toolchains/sega/m68k-elf/lib/gcc/m68k-elf/4.6.2/libgcc.a(xfgnulib.o)
 .debug_aranges
                0x00000520       0x20 /opt/toolchains/sega/m68k-elf/m68k-elf/lib/libnosys.a(sbrk.o)

.debug_line     0x00000000     0x45b2
 .debug_line    0x00000000      0x172 /opt/toolchains/sega/m68k-elf/m68k-elf/lib/libc.a(lib_a-malloc.o)
 .debug_line    0x00000172      0x31e /opt/toolchains/sega/m68k-elf/m68k-elf/lib/libc.a(lib_a-mallocr.o)
 .debug_line    0x00000490      0x12f /opt/toolchains/sega/m68k-elf/m68k-elf/lib/libc.a(lib_a-memcmp.o)
 .debug_line    0x000005bf       0x91 /opt/toolchains/sega/m68k-elf/m68k-elf/lib/libc.a(lib_a-memcpy.o)
 .debug_line    0x00000650       0x95 /opt/toolchains/sega/m68k-elf/m68k-elf/lib/libc.a(lib_a-memset.o)
 .debug_line    0x000006e5      0x11d /opt/toolchains/sega/m68k-elf/m68k-elf/lib/libc.a(lib_a-mlock.o)
 .debug_line    0x00000802      0x172 /opt/toolchains/sega/m68k-elf/m68k-elf/lib/libc.a(lib_a-rand.o)
 .debug_line    0x00000974      0x173 /opt/toolchains/sega/m68k-elf/m68k-elf/lib/libc.a(lib_a-sbrkr.o)
 .debug_line    0x00000ae7      0x189 /opt/toolchains/sega/m68k-elf/m68k-elf/lib/libc.a(lib_a-sprintf.o)
 .debug_line    0x00000c70       0xe6 /opt/toolchains/sega/m68k-elf/m68k-elf/lib/libc.a(lib_a-strcat.o)
 .debug_line    0x00000d56       0xc6 /opt/toolchains/sega/m68k-elf/m68k-elf/lib/libc.a(lib_a-strcpy.o)
 .debug_line    0x00000e1c      0x110 /opt/toolchains/sega/m68k-elf/m68k-elf/lib/libc.a(lib_a-strlen.o)
 .debug_line    0x00000f2c      0x12a /opt/toolchains/sega/m68k-elf/m68k-elf/lib/libc.a(lib_a-strncpy.o)
 .debug_line    0x00001056      0x8b4 /opt/toolchains/sega/m68k-elf/m68k-elf/lib/libc.a(lib_a-svfprintf.o)
 .debug_line    0x0000190a      0x6e5 /opt/toolchains/sega/m68k-elf/m68k-elf/lib/libc.a(lib_a-dtoa.o)
 .debug_line    0x00001fef      0x1f7 /opt/toolchains/sega/m68k-elf/m68k-elf/lib/libc.a(lib_a-freer.o)
 .debug_line    0x000021e6      0x10b /opt/toolchains/sega/m68k-elf/m68k-elf/lib/libc.a(lib_a-impure.o)
 .debug_line    0x000022f1      0x1a6 /opt/toolchains/sega/m68k-elf/m68k-elf/lib/libc.a(lib_a-locale.o)
 .debug_line    0x00002497      0x13f /opt/toolchains/sega/m68k-elf/m68k-elf/lib/libc.a(lib_a-memchr.o)
 .debug_line    0x000025d6      0x4be /opt/toolchains/sega/m68k-elf/m68k-elf/lib/libc.a(lib_a-mprec.o)
 .debug_line    0x00002a94      0x164 /opt/toolchains/sega/m68k-elf/m68k-elf/lib/libc.a(lib_a-reent.o)
 .debug_line    0x00002bf8      0x17c /opt/toolchains/sega/m68k-elf/m68k-elf/lib/libc.a(lib_a-s_fpclassify.o)
 .debug_line    0x00002d74       0xf9 /opt/toolchains/sega/m68k-elf/m68k-elf/lib/libc.a(lib_a-strcmp.o)
 .debug_line    0x00002e6d      0x5a9 /opt/toolchains/sega/m68k-elf/m68k-elf/lib/libc.a(lib_a-svfiprintf.o)
 .debug_line    0x00003416      0x14d /opt/toolchains/sega/m68k-elf/m68k-elf/lib/libc.a(lib_a-callocr.o)
 .debug_line    0x00003563      0x160 /opt/toolchains/sega/m68k-elf/m68k-elf/lib/libc.a(lib_a-memmove.o)
 .debug_line    0x000036c3      0x2c4 /opt/toolchains/sega/m68k-elf/m68k-elf/lib/libc.a(lib_a-reallocr.o)
 .debug_line    0x00003987       0x73 /opt/toolchains/sega/m68k-elf/lib/gcc/m68k-elf/4.6.2/libgcc.a(_mulsi3.o)
 .debug_line    0x000039fa       0x8c /opt/toolchains/sega/m68k-elf/lib/gcc/m68k-elf/4.6.2/libgcc.a(_udivsi3.o)
 .debug_line    0x00003a86       0x7b /opt/toolchains/sega/m68k-elf/lib/gcc/m68k-elf/4.6.2/libgcc.a(_divsi3.o)
 .debug_line    0x00003b01       0x77 /opt/toolchains/sega/m68k-elf/lib/gcc/m68k-elf/4.6.2/libgcc.a(_umodsi3.o)
 .debug_line    0x00003b78       0x77 /opt/toolchains/sega/m68k-elf/lib/gcc/m68k-elf/4.6.2/libgcc.a(_modsi3.o)
 .debug_line    0x00003bef      0x3ea /opt/toolchains/sega/m68k-elf/lib/gcc/m68k-elf/4.6.2/libgcc.a(_double.o)
 .debug_line    0x00003fd9       0x82 /opt/toolchains/sega/m68k-elf/lib/gcc/m68k-elf/4.6.2/libgcc.a(_floatex.o)
 .debug_line    0x0000405b       0x71 /opt/toolchains/sega/m68k-elf/lib/gcc/m68k-elf/4.6.2/libgcc.a(_eqdf2.o)
 .debug_line    0x000040cc       0x71 /opt/toolchains/sega/m68k-elf/lib/gcc/m68k-elf/4.6.2/libgcc.a(_nedf2.o)
 .debug_line    0x0000413d       0x71 /opt/toolchains/sega/m68k-elf/lib/gcc/m68k-elf/4.6.2/libgcc.a(_gtdf2.o)
 .debug_line    0x000041ae       0x71 /opt/toolchains/sega/m68k-elf/lib/gcc/m68k-elf/4.6.2/libgcc.a(_gedf2.o)
 .debug_line    0x0000421f       0x71 /opt/toolchains/sega/m68k-elf/lib/gcc/m68k-elf/4.6.2/libgcc.a(_ltdf2.o)
 .debug_line    0x00004290       0x6d /opt/toolchains/sega/m68k-elf/lib/gcc/m68k-elf/4.6.2/libgcc.a(_muldi3.o)
 .debug_line    0x000042fd      0x159 /opt/toolchains/sega/m68k-elf/lib/gcc/m68k-elf/4.6.2/libgcc.a(fpgnulib.o)
 .debug_line    0x00004456       0xf4 /opt/toolchains/sega/m68k-elf/lib/gcc/m68k-elf/4.6.2/libgcc.a(xfgnulib.o)
 .debug_line    0x0000454a       0x68 /opt/toolchains/sega/m68k-elf/m68k-elf/lib/libnosys.a(sbrk.o)

.debug_str      0x00000000     0x176b
 .debug_str     0x00000000      0x47b /opt/toolchains/sega/m68k-elf/m68k-elf/lib/libc.a(lib_a-malloc.o)
                                0x504 (size before relaxing)
 .debug_str     0x0000047b      0x206 /opt/toolchains/sega/m68k-elf/m68k-elf/lib/libc.a(lib_a-mallocr.o)
                                0x6d9 (size before relaxing)
 .debug_str     0x00000681       0x9c /opt/toolchains/sega/m68k-elf/m68k-elf/lib/libc.a(lib_a-memcmp.o)
                                0x138 (size before relaxing)
 .debug_str     0x0000071d       0x6b /opt/toolchains/sega/m68k-elf/m68k-elf/lib/libc.a(lib_a-mlock.o)
                                0x50b (size before relaxing)
 .debug_str     0x00000788       0x3d /opt/toolchains/sega/m68k-elf/m68k-elf/lib/libc.a(lib_a-rand.o)
                                0x4f3 (size before relaxing)
 .debug_str     0x000007c5       0xae /opt/toolchains/sega/m68k-elf/m68k-elf/lib/libc.a(lib_a-sbrkr.o)
                                0x4f8 (size before relaxing)
 .debug_str     0x00000873       0xc8 /opt/toolchains/sega/m68k-elf/m68k-elf/lib/libc.a(lib_a-sprintf.o)
                                0x525 (size before relaxing)
 .debug_str     0x0000093b       0x4b /opt/toolchains/sega/m68k-elf/m68k-elf/lib/libc.a(lib_a-strcat.o)
                                0x13c (size before relaxing)
 .debug_str     0x00000986       0xb0 /opt/toolchains/sega/m68k-elf/m68k-elf/lib/libc.a(lib_a-strcpy.o)
                                0x145 (size before relaxing)
 .debug_str     0x00000a36       0x49 /opt/toolchains/sega/m68k-elf/m68k-elf/lib/libc.a(lib_a-strlen.o)
                                0x147 (size before relaxing)
 .debug_str     0x00000a7f       0x64 /opt/toolchains/sega/m68k-elf/m68k-elf/lib/libc.a(lib_a-strncpy.o)
                                0x162 (size before relaxing)
 .debug_str     0x00000ae3      0x1a9 /opt/toolchains/sega/m68k-elf/m68k-elf/lib/libc.a(lib_a-svfprintf.o)
                                0x6d0 (size before relaxing)
 .debug_str     0x00000c8c      0x100 /opt/toolchains/sega/m68k-elf/m68k-elf/lib/libc.a(lib_a-dtoa.o)
                                0x5e9 (size before relaxing)
 .debug_str     0x00000d8c       0x3c /opt/toolchains/sega/m68k-elf/m68k-elf/lib/libc.a(lib_a-freer.o)
                                0x62b (size before relaxing)
 .debug_str     0x00000dc8       0x57 /opt/toolchains/sega/m68k-elf/m68k-elf/lib/libc.a(lib_a-impure.o)
                                0x502 (size before relaxing)
 .debug_str     0x00000e1f      0x270 /opt/toolchains/sega/m68k-elf/m68k-elf/lib/libc.a(lib_a-locale.o)
                                0x758 (size before relaxing)
 .debug_str     0x0000108f       0x53 /opt/toolchains/sega/m68k-elf/m68k-elf/lib/libc.a(lib_a-memchr.o)
                                0x152 (size before relaxing)
 .debug_str     0x000010e2       0xf6 /opt/toolchains/sega/m68k-elf/m68k-elf/lib/libc.a(lib_a-mprec.o)
                                0x5f6 (size before relaxing)
 .debug_str     0x000011d8       0x71 /opt/toolchains/sega/m68k-elf/m68k-elf/lib/libc.a(lib_a-reent.o)
                                0x527 (size before relaxing)
 .debug_str     0x00001249       0xcb /opt/toolchains/sega/m68k-elf/m68k-elf/lib/libc.a(lib_a-s_fpclassify.o)
                                0x18a (size before relaxing)
 .debug_str     0x00001314       0x40 /opt/toolchains/sega/m68k-elf/m68k-elf/lib/libc.a(lib_a-strcmp.o)
                                0x131 (size before relaxing)
 .debug_str     0x00001354       0x29 /opt/toolchains/sega/m68k-elf/m68k-elf/lib/libc.a(lib_a-svfiprintf.o)
                                0x643 (size before relaxing)
 .debug_str     0x0000137d       0x19 /opt/toolchains/sega/m68k-elf/m68k-elf/lib/libc.a(lib_a-callocr.o)
                                0x52a (size before relaxing)
 .debug_str     0x00001396       0x4b /opt/toolchains/sega/m68k-elf/m68k-elf/lib/libc.a(lib_a-memmove.o)
                                0x16b (size before relaxing)
 .debug_str     0x000013e1       0x59 /opt/toolchains/sega/m68k-elf/m68k-elf/lib/libc.a(lib_a-reallocr.o)
                                0x5ab (size before relaxing)
 .debug_str     0x0000143a       0xd6 /opt/toolchains/sega/m68k-elf/lib/gcc/m68k-elf/4.6.2/libgcc.a(_muldi3.o)
                                0x186 (size before relaxing)
 .debug_str     0x00001510       0xbc /opt/toolchains/sega/m68k-elf/lib/gcc/m68k-elf/4.6.2/libgcc.a(fpgnulib.o)
                                0x15f (size before relaxing)
 .debug_str     0x000015cc      0x103 /opt/toolchains/sega/m68k-elf/lib/gcc/m68k-elf/4.6.2/libgcc.a(xfgnulib.o)
                                0x1a7 (size before relaxing)
 .debug_str     0x000016cf       0x9c /opt/toolchains/sega/m68k-elf/m68k-elf/lib/libnosys.a(sbrk.o)
                                 0xc0 (size before relaxing)

.debug_frame    0x00000000      0xba4
 .debug_frame   0x00000000       0x4c /opt/toolchains/sega/m68k-elf/m68k-elf/lib/libc.a(lib_a-malloc.o)
 .debug_frame   0x0000004c       0x58 /opt/toolchains/sega/m68k-elf/m68k-elf/lib/libc.a(lib_a-mallocr.o)
 .debug_frame   0x000000a4       0x34 /opt/toolchains/sega/m68k-elf/m68k-elf/lib/libc.a(lib_a-memcmp.o)
 .debug_frame   0x000000d8       0x44 /opt/toolchains/sega/m68k-elf/m68k-elf/lib/libc.a(lib_a-mlock.o)
 .debug_frame   0x0000011c       0x4c /opt/toolchains/sega/m68k-elf/m68k-elf/lib/libc.a(lib_a-rand.o)
 .debug_frame   0x00000168       0x30 /opt/toolchains/sega/m68k-elf/m68k-elf/lib/libc.a(lib_a-sbrkr.o)
 .debug_frame   0x00000198       0x4c /opt/toolchains/sega/m68k-elf/m68k-elf/lib/libc.a(lib_a-sprintf.o)
 .debug_frame   0x000001e4       0x34 /opt/toolchains/sega/m68k-elf/m68k-elf/lib/libc.a(lib_a-strcat.o)
 .debug_frame   0x00000218       0x2c /opt/toolchains/sega/m68k-elf/m68k-elf/lib/libc.a(lib_a-strcpy.o)
 .debug_frame   0x00000244       0x2c /opt/toolchains/sega/m68k-elf/m68k-elf/lib/libc.a(lib_a-strlen.o)
 .debug_frame   0x00000270       0x34 /opt/toolchains/sega/m68k-elf/m68k-elf/lib/libc.a(lib_a-strncpy.o)
 .debug_frame   0x000002a4       0x9c /opt/toolchains/sega/m68k-elf/m68k-elf/lib/libc.a(lib_a-svfprintf.o)
 .debug_frame   0x00000340      0x158 /opt/toolchains/sega/m68k-elf/m68k-elf/lib/libc.a(lib_a-dtoa.o)
 .debug_frame   0x00000498       0x74 /opt/toolchains/sega/m68k-elf/m68k-elf/lib/libc.a(lib_a-freer.o)
 .debug_frame   0x0000050c       0xe0 /opt/toolchains/sega/m68k-elf/m68k-elf/lib/libc.a(lib_a-locale.o)
 .debug_frame   0x000005ec       0x34 /opt/toolchains/sega/m68k-elf/m68k-elf/lib/libc.a(lib_a-memchr.o)
 .debug_frame   0x00000620      0x2d4 /opt/toolchains/sega/m68k-elf/m68k-elf/lib/libc.a(lib_a-mprec.o)
 .debug_frame   0x000008f4       0x84 /opt/toolchains/sega/m68k-elf/m68k-elf/lib/libc.a(lib_a-reent.o)
 .debug_frame   0x00000978       0x2c /opt/toolchains/sega/m68k-elf/m68k-elf/lib/libc.a(lib_a-s_fpclassify.o)
 .debug_frame   0x000009a4       0x34 /opt/toolchains/sega/m68k-elf/m68k-elf/lib/libc.a(lib_a-strcmp.o)
 .debug_frame   0x000009d8       0x8c /opt/toolchains/sega/m68k-elf/m68k-elf/lib/libc.a(lib_a-svfiprintf.o)
 .debug_frame   0x00000a64       0x34 /opt/toolchains/sega/m68k-elf/m68k-elf/lib/libc.a(lib_a-callocr.o)
 .debug_frame   0x00000a98       0x38 /opt/toolchains/sega/m68k-elf/m68k-elf/lib/libc.a(lib_a-memmove.o)
 .debug_frame   0x00000ad0       0x68 /opt/toolchains/sega/m68k-elf/m68k-elf/lib/libc.a(lib_a-reallocr.o)
 .debug_frame   0x00000b38       0x40 /opt/toolchains/sega/m68k-elf/lib/gcc/m68k-elf/4.6.2/libgcc.a(_muldi3.o)
 .debug_frame   0x00000b78       0x2c /opt/toolchains/sega/m68k-elf/m68k-elf/lib/libnosys.a(sbrk.o)

.debug_ranges   0x00000000      0x428
 .debug_ranges  0x00000000       0x70 /opt/toolchains/sega/m68k-elf/m68k-elf/lib/libc.a(lib_a-mallocr.o)
 .debug_ranges  0x00000070       0x20 /opt/toolchains/sega/m68k-elf/m68k-elf/lib/libc.a(lib_a-strcat.o)
 .debug_ranges  0x00000090      0x168 /opt/toolchains/sega/m68k-elf/m68k-elf/lib/libc.a(lib_a-svfprintf.o)
 .debug_ranges  0x000001f8       0x18 /opt/toolchains/sega/m68k-elf/m68k-elf/lib/libc.a(lib_a-mprec.o)
 .debug_ranges  0x00000210       0x68 /opt/toolchains/sega/m68k-elf/m68k-elf/lib/libc.a(lib_a-svfiprintf.o)
 .debug_ranges  0x00000278       0x40 /opt/toolchains/sega/m68k-elf/m68k-elf/lib/libc.a(lib_a-callocr.o)
 .debug_ranges  0x000002b8      0x158 /opt/toolchains/sega/m68k-elf/m68k-elf/lib/libc.a(lib_a-reallocr.o)
 .debug_ranges  0x00000410       0x18 /opt/toolchains/sega/m68k-elf/lib/gcc/m68k-elf/4.6.2/libgcc.a(fpgnulib.o)
